Archive member included because of file (symbol)

c:/program files/atmel/winavr/bin/../lib/gcc/avr/4.3.0/avr5\libgcc.a(_exit.o)
                              c:/program files/atmel/winavr/bin/../lib/gcc/avr/4.3.0/../../../../avr/lib/avr5/crtm16.o (exit)
c:/program files/atmel/winavr/bin/../lib/gcc/avr/4.3.0/avr5\libgcc.a(_copy_data.o)
                              main.o (__do_copy_data)
c:/program files/atmel/winavr/bin/../lib/gcc/avr/4.3.0/avr5\libgcc.a(_clear_bss.o)
                              main.o (__do_clear_bss)
c:/program files/atmel/winavr/bin/../lib/gcc/avr/4.3.0/../../../../avr/lib/avr5\libc.a(strcpy.o)
                              main.o (strcpy)

Allocating common symbols
Common symbol       size              file

Receiv_int          0x1               Transceiver.o
ID_RX               0x1               Transceiver.o
x                   0x1               lcd_c.o
my_ID               0x1               Transceiver.o
Paket_in            0x10              Transceiver.o
Paket_out           0x10              Transceiver.o
y                   0x1               lcd_c.o

Memory Configuration

Name             Origin             Length             Attributes
text             0x00000000         0x00020000         xr
data             0x00800060         0x0000ffa0         rw !x
eeprom           0x00810000         0x00010000         rw !x
fuse             0x00820000         0x00000400         rw !x
lock             0x00830000         0x00000400         rw !x
signature        0x00840000         0x00000400         rw !x
*default*        0x00000000         0xffffffff

Linker script and memory map

LOAD c:/program files/atmel/winavr/bin/../lib/gcc/avr/4.3.0/../../../../avr/lib/avr5/crtm16.o
LOAD main.o
LOAD Transceiver.o
LOAD lcd_c.o
LOAD c:/program files/atmel/winavr/bin/../lib/gcc/avr/4.3.0/avr5\libgcc.a
LOAD c:/program files/atmel/winavr/bin/../lib/gcc/avr/4.3.0/../../../../avr/lib/avr5\libc.a
LOAD c:/program files/atmel/winavr/bin/../lib/gcc/avr/4.3.0/avr5\libgcc.a

.hash
 *(.hash)

.dynsym
 *(.dynsym)

.dynstr
 *(.dynstr)

.gnu.version
 *(.gnu.version)

.gnu.version_d
 *(.gnu.version_d)

.gnu.version_r
 *(.gnu.version_r)

.rel.init
 *(.rel.init)

.rela.init
 *(.rela.init)

.rel.text
 *(.rel.text)
 *(.rel.text.*)
 *(.rel.gnu.linkonce.t*)

.rela.text
 *(.rela.text)
 *(.rela.text.*)
 *(.rela.gnu.linkonce.t*)

.rel.fini
 *(.rel.fini)

.rela.fini
 *(.rela.fini)

.rel.rodata
 *(.rel.rodata)
 *(.rel.rodata.*)
 *(.rel.gnu.linkonce.r*)

.rela.rodata
 *(.rela.rodata)
 *(.rela.rodata.*)
 *(.rela.gnu.linkonce.r*)

.rel.data
 *(.rel.data)
 *(.rel.data.*)
 *(.rel.gnu.linkonce.d*)

.rela.data
 *(.rela.data)
 *(.rela.data.*)
 *(.rela.gnu.linkonce.d*)

.rel.ctors
 *(.rel.ctors)

.rela.ctors
 *(.rela.ctors)

.rel.dtors
 *(.rel.dtors)

.rela.dtors
 *(.rela.dtors)

.rel.got
 *(.rel.got)

.rela.got
 *(.rela.got)

.rel.bss
 *(.rel.bss)

.rela.bss
 *(.rela.bss)

.rel.plt
 *(.rel.plt)

.rela.plt
 *(.rela.plt)

.text           0x00000000      0x8a6
 *(.vectors)
 .vectors       0x00000000       0x54 c:/program files/atmel/winavr/bin/../lib/gcc/avr/4.3.0/../../../../avr/lib/avr5/crtm16.o
                0x00000000                __vectors
                0x00000000                __vector_default
 *(.vectors)
 *(.progmem.gcc*)
 *(.progmem*)
                0x00000054                . = ALIGN (0x2)
                0x00000054                __trampolines_start = .
 *(.trampolines)
 .trampolines   0x00000054        0x0 linker stubs
 *(.trampolines*)
                0x00000054                __trampolines_end = .
 *(.jumptables)
 *(.jumptables*)
 *(.lowtext)
 *(.lowtext*)
                0x00000054                __ctors_start = .
 *(.ctors)
                0x00000054                __ctors_end = .
                0x00000054                __dtors_start = .
 *(.dtors)
                0x00000054                __dtors_end = .
 SORT(*)(.ctors)
 SORT(*)(.dtors)
 *(.init0)
 .init0         0x00000054        0x0 c:/program files/atmel/winavr/bin/../lib/gcc/avr/4.3.0/../../../../avr/lib/avr5/crtm16.o
                0x00000054                __init
 *(.init0)
 *(.init1)
 *(.init1)
 *(.init2)
 .init2         0x00000054        0xc c:/program files/atmel/winavr/bin/../lib/gcc/avr/4.3.0/../../../../avr/lib/avr5/crtm16.o
 *(.init2)
 *(.init3)
 *(.init3)
 *(.init4)
 .init4         0x00000060       0x16 c:/program files/atmel/winavr/bin/../lib/gcc/avr/4.3.0/avr5\libgcc.a(_copy_data.o)
                0x00000060                __do_copy_data
 .init4         0x00000076       0x10 c:/program files/atmel/winavr/bin/../lib/gcc/avr/4.3.0/avr5\libgcc.a(_clear_bss.o)
                0x00000076                __do_clear_bss
 *(.init4)
 *(.init5)
 *(.init5)
 *(.init6)
 *(.init6)
 *(.init7)
 *(.init7)
 *(.init8)
 *(.init8)
 *(.init9)
 .init9         0x00000086        0x8 c:/program files/atmel/winavr/bin/../lib/gcc/avr/4.3.0/../../../../avr/lib/avr5/crtm16.o
 *(.init9)
 *(.text)
 .text          0x0000008e        0x4 c:/program files/atmel/winavr/bin/../lib/gcc/avr/4.3.0/../../../../avr/lib/avr5/crtm16.o
                0x0000008e                __vector_1
                0x0000008e                __vector_12
                0x0000008e                __bad_interrupt
                0x0000008e                __vector_6
                0x0000008e                __vector_3
                0x0000008e                __vector_11
                0x0000008e                __vector_13
                0x0000008e                __vector_17
                0x0000008e                __vector_19
                0x0000008e                __vector_7
                0x0000008e                __vector_5
                0x0000008e                __vector_4
                0x0000008e                __vector_9
                0x0000008e                __vector_15
                0x0000008e                __vector_8
                0x0000008e                __vector_14
                0x0000008e                __vector_10
                0x0000008e                __vector_16
                0x0000008e                __vector_20
 .text          0x00000092      0x116 main.o
                0x0000010a                main
                0x00000092                __vector_2
 .text          0x000001a8      0x55e Transceiver.o
                0x00000352                Init_RF
                0x000002ac                receive_mode
                0x000001b2                Start_SPI
                0x00000288                rf_sleep
                0x000001c0                Start_SPI_soft
                0x000002be                FIFO_reset
                0x000002e0                Low_power
                0x0000029a                transmit_mode
                0x00000266                Clr_VDI
                0x000001d8                Write_cmd
                0x000005e0                Send_data
                0x000003c4                Init_Transceiver
                0x000001a8                delay
                0x00000432                Send_paket
                0x000002d0                Write_FSK
                0x0000065c                Receiv_data
                0x00000532                Receiv_paket
                0x000001ca                Start_Inter
                0x00000696                __vector_18
                0x00000234                Rx_FIFO
 .text          0x00000706      0x18e lcd_c.o
                0x00000748                lcd_data
                0x00000706                lcd_write
                0x000007a6                lcd_gotoxy
                0x00000802                lcd_newline
                0x00000816                lcd_putc
                0x00000758                lcd_clrscr
                0x00000856                lcd_puts
                0x00000770                lcd_init
                0x000007d6                lcd_secondline
                0x0000086e                lcd_firstline
                0x00000750                lcd_command
                0x0000079a                toggle_e
 .text          0x00000894        0x0 c:/program files/atmel/winavr/bin/../lib/gcc/avr/4.3.0/avr5\libgcc.a(_exit.o)
 .text          0x00000894        0x0 c:/program files/atmel/winavr/bin/../lib/gcc/avr/4.3.0/avr5\libgcc.a(_copy_data.o)
 .text          0x00000894        0x0 c:/program files/atmel/winavr/bin/../lib/gcc/avr/4.3.0/avr5\libgcc.a(_clear_bss.o)
 .text          0x00000894        0xe c:/program files/atmel/winavr/bin/../lib/gcc/avr/4.3.0/../../../../avr/lib/avr5\libc.a(strcpy.o)
                0x00000894                strcpy
                0x000008a2                . = ALIGN (0x2)
 *(.text.*)
 .text.libgcc   0x000008a2        0x0 c:/program files/atmel/winavr/bin/../lib/gcc/avr/4.3.0/avr5\libgcc.a(_exit.o)
 .text.libgcc   0x000008a2        0x0 c:/program files/atmel/winavr/bin/../lib/gcc/avr/4.3.0/avr5\libgcc.a(_copy_data.o)
 .text.libgcc   0x000008a2        0x0 c:/program files/atmel/winavr/bin/../lib/gcc/avr/4.3.0/avr5\libgcc.a(_clear_bss.o)
                0x000008a2                . = ALIGN (0x2)
 *(.fini9)
 .fini9         0x000008a2        0x0 c:/program files/atmel/winavr/bin/../lib/gcc/avr/4.3.0/avr5\libgcc.a(_exit.o)
                0x000008a2                exit
                0x000008a2                _exit
 *(.fini9)
 *(.fini8)
 *(.fini8)
 *(.fini7)
 *(.fini7)
 *(.fini6)
 *(.fini6)
 *(.fini5)
 *(.fini5)
 *(.fini4)
 *(.fini4)
 *(.fini3)
 *(.fini3)
 *(.fini2)
 *(.fini2)
 *(.fini1)
 *(.fini1)
 *(.fini0)
 .fini0         0x000008a2        0x4 c:/program files/atmel/winavr/bin/../lib/gcc/avr/4.3.0/avr5\libgcc.a(_exit.o)
 *(.fini0)
                0x000008a6                _etext = .

.data           0x00800060       0x1c load address 0x000008a6
                0x00800060                PROVIDE (__data_start, .)
 *(.data)
 .data          0x00800060        0x0 c:/program files/atmel/winavr/bin/../lib/gcc/avr/4.3.0/../../../../avr/lib/avr5/crtm16.o
 .data          0x00800060        0xb main.o
 .data          0x0080006b        0x0 Transceiver.o
 .data          0x0080006b       0x11 lcd_c.o
 .data          0x0080007c        0x0 c:/program files/atmel/winavr/bin/../lib/gcc/avr/4.3.0/avr5\libgcc.a(_exit.o)
 .data          0x0080007c        0x0 c:/program files/atmel/winavr/bin/../lib/gcc/avr/4.3.0/avr5\libgcc.a(_copy_data.o)
 .data          0x0080007c        0x0 c:/program files/atmel/winavr/bin/../lib/gcc/avr/4.3.0/avr5\libgcc.a(_clear_bss.o)
 .data          0x0080007c        0x0 c:/program files/atmel/winavr/bin/../lib/gcc/avr/4.3.0/../../../../avr/lib/avr5\libc.a(strcpy.o)
 *(.data*)
 *(.rodata)
 *(.rodata*)
 *(.gnu.linkonce.d*)
                0x0080007c                . = ALIGN (0x2)
                0x0080007c                _edata = .
                0x0080007c                PROVIDE (__data_end, .)

.bss            0x0080007c       0x25 load address 0x000008c2
                0x0080007c                PROVIDE (__bss_start, .)
 *(.bss)
 .bss           0x0080007c        0x0 c:/program files/atmel/winavr/bin/../lib/gcc/avr/4.3.0/../../../../avr/lib/avr5/crtm16.o
 .bss           0x0080007c        0x0 main.o
 .bss           0x0080007c        0x0 Transceiver.o
 .bss           0x0080007c        0x0 lcd_c.o
 .bss           0x0080007c        0x0 c:/program files/atmel/winavr/bin/../lib/gcc/avr/4.3.0/avr5\libgcc.a(_exit.o)
 .bss           0x0080007c        0x0 c:/program files/atmel/winavr/bin/../lib/gcc/avr/4.3.0/avr5\libgcc.a(_copy_data.o)
 .bss           0x0080007c        0x0 c:/program files/atmel/winavr/bin/../lib/gcc/avr/4.3.0/avr5\libgcc.a(_clear_bss.o)
 .bss           0x0080007c        0x0 c:/program files/atmel/winavr/bin/../lib/gcc/avr/4.3.0/../../../../avr/lib/avr5\libc.a(strcpy.o)
 *(.bss*)
 *(COMMON)
 COMMON         0x0080007c       0x23 Transceiver.o
                0x0080007c                Receiv_int
                0x0080007d                ID_RX
                0x0080007e                my_ID
                0x0080007f                Paket_in
                0x0080008f                Paket_out
 COMMON         0x0080009f        0x2 lcd_c.o
                0x0080009f                x
                0x008000a0                y
                0x008000a1                PROVIDE (__bss_end, .)
                0x000008a6                __data_load_start = LOADADDR (.data)
                0x000008c2                __data_load_end = (__data_load_start + SIZEOF (.data))

.noinit         0x008000a1        0x0
                0x008000a1                PROVIDE (__noinit_start, .)
 *(.noinit*)
                0x008000a1                PROVIDE (__noinit_end, .)
                0x008000a1                _end = .
                0x008000a1                PROVIDE (__heap_start, .)

.eeprom         0x00810000        0x0
 *(.eeprom*)
                0x00810000                __eeprom_end = .

.fuse
 *(.fuse)
 *(.lfuse)
 *(.hfuse)
 *(.efuse)

.lock
 *(.lock*)

.signature
 *(.signature*)

.stab
 *(.stab)

.stabstr
 *(.stabstr)

.stab.excl
 *(.stab.excl)

.stab.exclstr
 *(.stab.exclstr)

.stab.index
 *(.stab.index)

.stab.indexstr
 *(.stab.indexstr)

.comment
 *(.comment)

.debug
 *(.debug)

.line
 *(.line)

.debug_srcinfo
 *(.debug_srcinfo)

.debug_sfnames
 *(.debug_sfnames)

.debug_aranges  0x00000000       0x60
 *(.debug_aranges)
 .debug_aranges
                0x00000000       0x20 main.o
 .debug_aranges
                0x00000020       0x20 Transceiver.o
 .debug_aranges
                0x00000040       0x20 lcd_c.o

.debug_pubnames
                0x00000000      0x275
 *(.debug_pubnames)
 .debug_pubnames
                0x00000000       0x2a main.o
 .debug_pubnames
                0x0000002a      0x17b Transceiver.o
 .debug_pubnames
                0x000001a5       0xd0 lcd_c.o

.debug_info     0x00000000      0xb1f
 *(.debug_info)
 .debug_info    0x00000000      0x157 main.o
 .debug_info    0x00000157      0x677 Transceiver.o
 .debug_info    0x000007ce      0x351 lcd_c.o
 *(.gnu.linkonce.wi.*)

.debug_abbrev   0x00000000      0x4ac
 *(.debug_abbrev)
 .debug_abbrev  0x00000000       0xc1 main.o
 .debug_abbrev  0x000000c1      0x280 Transceiver.o
 .debug_abbrev  0x00000341      0x16b lcd_c.o

.debug_line     0x00000000      0xdc9
 *(.debug_line)
 .debug_line    0x00000000      0x181 main.o
 .debug_line    0x00000181      0x880 Transceiver.o
 .debug_line    0x00000a01      0x3c8 lcd_c.o

.debug_frame    0x00000000      0x250
 *(.debug_frame)
 .debug_frame   0x00000000       0x30 main.o
 .debug_frame   0x00000030      0x150 Transceiver.o
 .debug_frame   0x00000180       0xd0 lcd_c.o

.debug_str      0x00000000      0x2e7
 *(.debug_str)
 .debug_str     0x00000000       0xdb main.o
                                0x114 (size before relaxing)
 .debug_str     0x000000db      0x17a Transceiver.o
                                0x274 (size before relaxing)
 .debug_str     0x00000255       0x92 lcd_c.o
                                0x16f (size before relaxing)

.debug_loc      0x00000000      0x3b5
 *(.debug_loc)
 .debug_loc     0x00000000      0x277 Transceiver.o
 .debug_loc     0x00000277      0x13e lcd_c.o

.debug_macinfo
 *(.debug_macinfo)
OUTPUT(Transceiver.elf elf32-avr)
LOAD linker stubs
